:107E0000112484B714BE81FF0E94EE3F82E080936C
:107E1000C00088E18093C10096E09093C20090E199
:107E20009093C400809360008EE080936000C0E077
:107E3000D0E008E128E0F22EEE24E39435E0D32EE2
:107E400041E1C42E13E00E94CB3F813489F40E94AB
:107E5000CB3FB82E0E94D73F82E8B81621F1E1E867
:107E6000BE1202C085E001C083E00E94C43F88C00A
:107E7000823411F484E103C0853421F485E00E944A
:107E8000E53F7EC0853551F40E94CB3FC82F0E944C
:107E9000CB3FD0E0D82BCC0FDD1F70C0863529F446
:107EA00084E00E94E53F80E0E0CF843609F040C0E6
:107EB0000E94CB3F0E94CB3F982E0E94CB3FC11522
:107EC000F0E7DF0718F4FE0117BFE895A12CBB24EB
:107ED000B3940E94CB3FF50181935F019E12F9CFCD
:107EE000C115F0E7DF0718F0FE0117BFE8950E9403
:107EF000D73F07B600FCFDCFFE01A0E0B1E08C91BA
:107F000011962C91119790E0922B0C01E7BEE89509
:107F1000112432961296A03881E0B80781F7FE014D
:107F2000D7BEE89507B600FCFDCFC7BEE89528C0D0
:107F3000843791F40E94CB3F0E94CB3FB82E0E9421
:107F4000CB3F0E94D73FFE018591EF010E94C43FC5
:107F5000BA94B110F8CF14C0853751F40E94D73FBE
:107F60008EE10E94C43F85E90E94C43F86E17DCF37
:107F7000813521F400936000F09260000E94D73FA9
:107F800080E10E94C43F5FCF9091C00095FFFCCF7D
:107F90008093C60008958091C00087FFFCCF809138
:107FA000C00084FD01C0A8958091C60008950E947C
:107FB000CB3F803239F088E18093600088E0809385
:107FC0006000FFCF84E10C94C43FCF93C82F0E9480
:107FD000CB3FC150E1F7CF910C94D73F282EE0E67C
:0E7FE000F0E088E180831082EE27FF270994ED
:0400000300007E007B
:00000001FF
